:100000000C942A000C9447000C9447000C94470071
:100010000C9447000C9447000C9449000C94470042
:100020000C9447000C9447000C9447000C94470034
:100030000C9447000C9447000C9447000C94470024
:100040000C9447000C9447000C9447000C94470014
:100050000C94470011241FBECFE5D8E0DEBFCDBF12
:1000600010E0A0E6B0E0E0E3FAE002C005900D92F7
:10007000A837B107D9F710E0A8E7B0E001C01D929A
:10008000AC37B107E1F70E946D000C9416050C9493
:1000900000001F920F920FB60F9211242F933F93DF
:1000A0008F939F9386B597B5209178003091790012
:1000B000821B930B90937B0080937A0086B597B553
:1000C00090937900809378009F918F913F912F9129
:1000D0000F900FBE0F901F9018956F927F928F9286
:1000E0009F92AF92BF92CF92DF92EF92FF920F93C7
:1000F0001F93DF93CF93CDB7DEB761970FB6F89418
:10010000DEBF0FBECDBF8FEF87BB88BB0E949801BB
:1001100080E060E00E948F0180E88FBD81E08EBDAD
:100120001DBC1CBC80E289BF789480E690E00E94F0
:10013000F40120E030E0612C4AE5742E6E01089451
:10014000C11CD11C91E1892E912C81E7A82E80E061
:10015000B82EE0907A00F0907B000DC0F30131974B
:10016000F1F701968A309105C8F388B3805888BBAF
:10017000E216F30619F480E090E0F4CF81E060E04D
:100180000E94D0018DB79EB708970FB6F8949EBF16
:100190000FBE8DBF0DB71EB70F5F1F4FEDB7FEB778
:1001A000D282C182F80193828282B582A482209198
:1001B0007A0030917B0040E050E060E070E488E33A
:1001C00090E00E940F02F801378326830E943102DB
:1001D0008DB79EB708960FB6F8949EBF0FBE8DBF21
:1001E000C6010E94F4019701B4CF8150F0F7089541
:1001F00081509040E8F708958AB38E608ABB8AB335
:100200008F708ABB8BB3846F8BBBDB9882E081508D
:10021000F0F7D99A81E08150F0F799B3907FD9989F
:1002200082E08150F0F7D99A81E08150F0F789B3EC
:10023000D99882958F70892B08958AB38E608ABB76
:100240008AB38F708ABB8BB38C6F8BBB82E081507B
:10025000F0F7D99A81E08150F0F799B3907FD9985F
:1002600082E08150F0F7D99A81E08150F0F789B3AC
:10027000D99882958F70892B08950E94FC0087FD84
:10028000FCCF089582E08150F0F7D99A81E0815047
:10029000F0F7D99808951F93182F0E943D018AB353
:1002A0008E6F8ABB8BB381708BBB9BB3812F807F9A
:1002B000892B8BBB0E9442018BB381708BBB8BB3AC
:1002C0001295107F812B8BBB0E9442011F910895D4
:1002D0001F93182F0E943D018AB38E6F8ABB8BB388
:1002E00081708BBB8BB38860912F907F892B8BBBE8
:1002F0000E9442018BB381708BBB8BB388601295D7
:10030000107F812B8BBB0E9442011F91089581E0D9
:100310000E944B01089582E00E944B0108958823BA
:1003200011F48CE001C08EE0860F0E944B0108950D
:100330008AB38E6F8ABB80E096E381509040E8F7E5
:100340008BB381708BBB8BB380638BBB0E944201EC
:1003500082EC9EE081509040E8F70E9442018CE5DB
:1003600090E081509040E8F70E9442018CE590E0D7
:1003700081509040E8F7DC980E9442018CE590E0C3
:1003800081509040E8F788E20E944B0186E00E948D
:100390004B010E94870181E061E00E948F01089576
:1003A000823060F4603150F490E0029626E0880FCD
:1003B000991F2A95E1F7860F0E944B0108950E942C
:1003C0003D010E94FC0090E036E0969587953A95B5
:1003D000E1F7817008950E943D010E94FC008F7337
:1003E00008950E9468010895CF93DF93EC0103C044
:1003F00021960E94680188818823D1F7DF91CF91EF
:100400000895CF93DF93EC0102C00E946801FE01C2
:10041000219684918823C9F7DF91CF910895A1E2B5
:100420001A2EAA1BBB1BFD010DC0AA1FBB1FEE1F6E
:10043000FF1FA217B307E407F50720F0A21BB30BB9
:10044000E40BF50B661F771F881F991F1A9469F735
:1004500060957095809590959B01AC01BD01CF0191
:100460000895AEE0B0E0E7E3F2E00C94ED040D890E
:100470001E898F89988D97FF02C080E090E80197D0
:100480009E838D831A83098386E08C839E01255E7B
:100490003F4FCE010196698D7A8DA9010E946202BB
:1004A0004D815E8157FD0AC02F8138854217530761
:1004B0000CF49A01020F131FF80110822E96E4E04B
:1004C0000C940905ABE0B0E0E8E6F2E00C94DF0440
:1004D0003C012B015A01FC0117821682838181FDA8
:1004E00003C06FEF7FEFC6C19AE0892E1E0108940A
:1004F000211C311CF3012381F20123FD859123FF8F
:1005000081912F01882309F4B2C1853239F423FD8A
:10051000859123FF81912F01853229F490E0B30169
:100520000E945504E7CF982FFF24EE249924FFE181
:10053000FF15D0F09B3269F09C3228F4903259F0CC
:10054000933291F40EC09D3249F0903369F441E04A
:1005500024C052E0F52A84E0F82A28C098E0F92A5D
:1005600025C0E0E1FE2A22C0F7FC29C0892F805374
:100570008A3070F4F6FE05C0989C902C1124980ED9
:1005800015C0E89CE02C1124E80EF0E2FF2A0EC012
:100590009E3229F4F6FC6BC140E4F42A07C09C3675
:1005A00019F450E8F52A02C0983649F4F20123FD07
:1005B000959123FF91912F01992309F0B8CF892FAD
:1005C0008554833018F08052833038F444E050E092
:1005D000A40EB51E5FE359830FC0933631F09337F5
:1005E00079F0933509F056C020C0F50180818983E8
:1005F00042E050E0A40EB51E610101E010E012C01F
:10060000F501C080D180F6FC03C06FEF7FEF02C020
:10061000692D70E042E050E0A40EB51EC6010E94B4
:100620004A048C015FE7F52214C0F501C080D18037
:10063000F6FC03C06FEF7FEF02C0692D70E042E06F
:1006400050E0A40EB51EC6010E943F048C0150E884
:10065000F52AF3FE07C01AC080E290E0B3010E94C1
:100660005504EA948E2D90E008171907A8F30EC0E0
:10067000F601F7FC8591F7FE81916F0190E0B301DF
:100680000E945504E110EA94015010400115110533
:1006900079F7EAC0943611F0993669F5F7FE08C08B
:1006A000F501208131814281538184E090E00AC0CC
:1006B000F501808191819C01442737FD4095542F9D
:1006C00082E090E0A80EB91E9FE6F92257FF09C00C
:1006D00050954095309521953F4F4F4F5F4FE0E843
:1006E000FE2ACA01B901A1012AE030E00E9481047A
:1006F000D82ED21840C0953729F41F2D1F7E2AE02E
:1007000030E01DC01F2D197F9F3661F0903720F417
:10071000983509F0ACC00FC0903739F0983709F020
:10072000A6C004C028E030E00AC0106114FD1460C7
:1007300020E130E004C014FD166020E132E017FF34
:1007400008C0F501608171818281938144E050E0AD
:1007500008C0F50180819181BC0180E090E042E019
:1007600050E0A40EB51EA1010E948104D82ED2181B
:100770008FE7F82EF122F6FE0BC05EEFF522D914BA
:1007800038F4F4FE07C0F2FC05C08FEEF82202C078
:100790001D2D01C0192DF4FE0DC0FE01ED0DF11D42
:1007A0008081803319F499EEF92208C01F5FF2FEB0
:1007B00005C003C08F2D867809F01F5F0F2DF3FC55
:1007C00014C0F0FE0FC01E1510F09D2C0BC09D2C08
:1007D0009E0C911A1E2D06C080E290E0B3010E948B
:1007E00055041F5F1E15C0F304C01E1510F4E11A56
:1007F00001C0EE2404FF0FC080E390E0B3010E942B
:10080000550402FF1DC001FD03C088E790E00EC043
:1008100088E590E00BC0802F867891F001FF02C040
:100820008BE201C080E2F7FC8DE290E0B3010E9410
:10083000550406C080E390E0B3010E9455049A94E9
:10084000D914C0F3DA94F101ED0DF11D808190E02F
:10085000B3010E945504DD20A9F706C080E290E0B4
:10086000B3010E945504EA94EE20C1F743CEF30190
:1008700066817781CB012B96E2E10C94FB04FC01AD
:100880000590615070400110D8F7809590958E0FBB
:100890009F1F0895FC016150704001900110D8F72E
:1008A000809590958E0F9F1F08950F931F93CF9360
:1008B000DF938C01EB018B8181FF1BC082FF0DC098
:1008C0002E813F818C819D812817390764F4E8814E
:1008D000F9810193F983E88306C0E885F985802FC3
:1008E0000995892B31F48E819F8101969F838E8398
:1008F00002C00FEF1FEFC801DF91CF911F910F9141
:100900000895FA01AA27283051F1203181F1E894A5
:100910006F936E7F6E5F7F4F8F4F9F4FAF4FB1E0F2
:100920003ED0B4E03CD0670F781F891F9A1FA11DED
:10093000680F791F8A1F911DA11D6A0F711D811DEE
:10094000911DA11D20D009F468943F912AE0269FB3
:1009500011243019305D3193DEF6CF010895462F12
:100960004770405D4193B3E00FD0C9F7F6CF462FF3
:100970004F70405D4A3318F0495D31FD405241935C
:1009800002D0A9F7EACFB4E0A69597958795779519
:100990006795BA95C9F700976105710508959B01A0
:1009A000AC010A2E06945795479537952795BA9529
:1009B000C9F7620F731F841F951FA01D08952F9202
:1009C0003F924F925F926F927F928F929F92AF92DF
:1009D000BF92CF92DF92EF92FF920F931F93CF932C
:1009E000DF93CDB7DEB7CA1BDB0B0FB6F894DEBFC3
:1009F0000FBECDBF09942A88398848885F846E84E9
:100A00007D848C849B84AA84B984C884DF80EE8032
:100A1000FD800C811B81AA81B981CE0FD11D0FB63B
:100A2000F894DEBF0FBECDBFED010895F894FFCF5F
:100A30004465206672657175656E746965206973B9
:080A40000025347520487A00FE
:00000001FF
